:020000040000FA
:1000000064008510831685017F30810083126400AF
:1000100085018C0120308D003A308E006400060886
:1000200003108E0703188D0A8C0A0A300C02031D78
:100030000E28FF308C0064008B218B218B218B21BB
:100040008B218B218B218B218B218B218B218B2150
:100050008B218B21051285158B2105168B218B2178
:1000600005128B2105168B218B218B2105128B21EB
:1000700005168B218C1F05168C1B05128B21051272
:100080008B218B218B218B2105168B2105128B2136
:1000900005168B21051285118B2100000000000040
:1000A00085158B218B218B2105168B2105128B2128
:1000B0008D1D05128D1905168B210D1D05120D19AB
:1000C00005168B218D1C05128D1805168B210D1C14
:1000D00005120D1805168B218E1F05128E1B051695
:1000E0008B210E1F05120E1B05168B218E1E05126D
:1000F0008E1A05168B210E1E05120E1A05168B215F
:100100008E1D05128E1905168B210E1D05120E1956
:1001100005168B218E1C05128E1805168B210512D3
:100120008B2185118B218C0A0000000000008C1DA2
:100130001B2885158B2105168B218B2105128B2100
:100140008B218B218B2105168B218B218B21051275
:100150008B218B218B218B2105168B2105128B2165
:1001600005168B21051285118B210000000000006F
:1001700085158B218B218B2105168B2105128B2157
:100180008D1D05128D1905168B210D1D05120D19DA
:1001900005168B218D1C05128D1805168B210D1C43
:1001A00005120D1805168B218E1F05128E1B0516C4
:1001B0008B210E1F05120E1B05168B218E1E05129C
:1001C0008E1A05168B210E1E05120E1A05168B218E
:1001D0008E1D05128E1905168B210E1D05120E1986
:1001E00005168B218E1C05128E1805168B21051203
:1001F0008B2185118B2185148F0190019101640061
:100200008F0A031D0629900A0319910A911EFF28DF
:10021000FF308C008B218B218B218B218B218B211B
:100220008B218B218B218B218B218B218B218B216E
:10023000051285158B2105168B218B2105128B212B
:1002400005128B218B218B2105168B2105168B2105
:100250008C1F05168C1B05128B2105128B218B21FF
:100260008B218B2105168B2105128B2105168B21E5
:10027000051285118B2100000000000085158B21DF
:100280008B218B2105168B2105128B218D1D0512CB
:100290008D1905168B210D1D05120D1905168B21C3
:1002A0008D1C05128D1805168B210D1C05120D18BD
:1002B00005168B218E1F05128E1B05168B210E1F16
:1002C00005120E1B05168B218E1E05128E1A0516A1
:1002D0008B210E1E05120E1A05168B218E1D05127E
:1002E0008E1905168B210E1D05120E1905168B2170
:1002F0008E1C05128E1805168B2105128B21851177
:100300008B210000000000008C0A8C1D0A298F013F
:0C03100090019101FF280515051108005F
:02400E00F73F7A
:00000001FF
